:020000000A28CC
:10000800FE00030EF2000A08F300C72F4F288312E0
:1000180003134208FF004108840000210038031937
:1000280008004208FF00410884000021D525C10AC4
:100038000319C20A64000B2883123708F500193027
:10004800F5078312031337087502F40074080319BF
:10005800080064002528F70083120313861686100B
:10006800770850278312031386140800F7008312B9
:1000780003138612861077085027831203138614F9
:1000880008008C2E912E962E9B2EA02EA52EAA2EE1
:10009800AF2EB42EB92E2030F001F1018313840065
:1000A8003A3061208301EA2BF90078080739403893
:1000B8003A2079087F3980383A2864008001840A18
:1000C800040603190034040662288A30F400F40B8D
:1000D8006B2808001230F400F40B702808009E30DA
:0800E800F400F40B7528080078
:10020000FF1B0A2983137F1883170008840A031928
:10021000FF0A08007F087F398A000408840A03194E
:10022000FF0A82000034003400340034003400340B
:1002300000345F34003400340034073400340734B1
:1002400000340034063409340934063424342A34A2
:100250007F342A341234233413340834643462343F
:1002600036344934553422345034003405340334A0
:100270000034003400341C3422344134003400345F
:10028000413422341C34003408342A341C342A34D7
:100290000834083408343E34083408340034503408
:1002A0003034003400340834083408340834083456
:1002B0000034303430340034003420341034083406
:1002C000043402343E345134493445343E3400342D
:1002D00042347F3440340034423461345134493440
:1002E00046342134413445344B34313418341434D9
:1002F00012347F341034273445344534453439348E
:100300003C344A344934493430340134713409348A
:1003100005340334363449344934493436340634E8
:100320004934493429341E340034363436340034E8
:100330000034003456343634003400340034083489
:100340001434223441341434143414341434143432
:10035000413422341434083400340234013451342A
:100360000934063432344934793441343E347E34ED
:100370001134113411347E347F34493449344934D2
:1003800036343E3441344134413422347F344134B4
:10039000413422341C347F344934493449344134A3
:1003A0007F3409340934013401343E34413441345A
:1003B000513432347F340834083408347F34003404
:1003C00041347F34413400342034403441343F34AC
:1003D00001347F3408341434223441347F344034BF
:1003E0004034403440347F340234043402347F34A7
:1003F0007F340434083410347F343E344134413483
:1004000041343E347F3409340934093406343E34EF
:100410004134513421345E347F3409341934293461
:100420004634463449344934493431340134013492
:100430007F34013401343F344034403440343F345D
:100440001F342034403420341F347F342034183497
:1004500020347F3463341434083414346334033464
:100460000434783404340334613451344934453429
:1004700043347E341134113411347E347F344534A6
:100480004534453439347F34493449344934363479
:100490007F340134013401340334C0347E344134B8
:1004A0007F34C0347F34493449344934413477345B
:1004B00008347F3408347734223449344934493499
:1004C00036347F342034103408347F347F34203481
:1004D000133408347F347F340834143422344134E4
:1004E00040343E34013401347F347F3402340434E8
:1004F00002347F347F340834083408347F343E3487
:100500004134413441343E347F34013401340134C8
:100510007F347F3409340934093406343E3441349D
:10052000413441342234013401347F340134013404
:1005300027344834483448343F341E3421347F341F
:1005400021341E34633414340834143463347F3457
:10055000403440347F34C0340F34103410341034FD
:100560007F347F3440347C3440347F347F344034B3
:100570007C344034FF3401347F34483448343034E0
:100580007F344834303400347F347F344834483446
:100590004834303422344934493449343E347F3489
:1005A00008343E3441343E34763409340934093455
:1005B0007F34203454345434543478347C345434B8
:1005C0005434543424347C3454345434543428341F
:1005D0007C340434043404340C34C034783444346B
:1005E0007C34C034383454345434543418346C3477
:1005F00010347C3410346C3428344434543454343F
:1006000028347C342034103408347C347C34213455
:10061000123408347C347C3410341034283444349C
:1006200040343834043404347C347C34083410349A
:1006300008347C347C341034103410347C34383436
:1006400044344434443438347C340434043404347E
:100650007C347C3414341434143408343834443442
:10066000443444342034043404347C3404340434B6
:100670000C345034503450343C34183424347C34EA
:1006800024341834443428341034283444347C342A
:10069000403440347C34C0340C34103410341034C2
:1006A0007C347C344034783440347C347C34403482
:1006B00078344034FC347C34543450345034203456
:1006C0007C345034203400347C347C345034503406
:1006D00050342034283444345434543438347C3442
:1006E0001034383444343834483434341434143402
:1006F0007C342034D234E534EC34EF34E534F03457
:10070000E034F234F334F034E0343A3420342D342D
:100710002D342D342D342D342D342D342D342D34D1
:100720002D342D342D342D342D3400342D342D34EE
:100730002D342D342D342D342D342D342D342D34B1
:100740002D342D342D342D34443453343134383455
:100750004234323430342034203456344E344E3423
:1007600049344B3400342034CE34E134F034FB349B
:10077000E2342034003420342034CA342E34C734D8
:100780002E3420340034D334EB34E834F634E034FF
:100790003A34003420342034C434EE34EC343A3467
:1007A00000342334433400342C34003430340034E7
:1007B00031340034323400343334003434340034CF
:1007C00035340034363400343734003438340034AF
:1007D0003934003464008F2770270030F801582026
:1007E0007930C1008330C2000B200230F8000030A5
:1007F0005820CA30C1008330C2000B200330F800FB
:1008000000305820C330C1008330C2000B200430B8
:10081000F800003058209630C1008330C2000B2011
:100820008B133B268B17831203132E030319872C7C
:100830002E08023A03197F2CCC308B132F278B17ED
:1008400071182A2C44308B132F278B1771148312A5
:10085000B8017111711C3A2C0130711D00398312DD
:10086000061D0039003803193A2CBE308B132F2790
:100870008B1770172020701F902C8B13EC2683127F
:100880000313B300EC2683120313B5008B17FA0091
:10089000330810250230711171107013F8002A30DE
:1008A00058202308C2002208C1000B202508C200DE
:1008B0002408C1000B202708C2002608C1000B2015
:1008C000B108031D712CB008031D712CB208031D63
:1008D000712C2B082A04031D712CB930C100833000
:1008E000742CD430C1008330C2000B202908C20010
:1008F0002808C1000B20D130C10083308E2C02307B
:10090000F8002A305820B330C10083308E2C0230DA
:10091000F8002A305820BB30C1008330C2000B20C1
:100920002F030319062D2F08023A0319FC2CCC3093
:100930008B130E278B17F118A52C44308B130E2721
:100940008B17F1148312B901F111F11CB52C013090
:10095000F11D00398312051E003900380319B52C2A
:10096000BE308B130E278B17F0172020F01FED2BB6
:100970008B13CA2683120313B400CA2683120313EF
:10098000B6008B17FA00340810250330F111F1106E
:10099000F013F8002A3058202308C2002208C100B2
:1009A0000B202508C2002408C1000B202708C20024
:1009B0002608C1000B20B108031DEC2CB008031D54
:1009C000EC2CB208031DEC2C2B082A04031DEC2C84
:1009D000B930C1008330EF2CD430C1008330C20065
:1009E0000B202908C2002808C1000B20D130C1000B
:1009F0008330C2000B20ED2B0330F8002A30582042
:100A0000B330C1008330C2000B20ED2B0330F8005F
:100A10002A305820BB30C1008330C2000B20ED2BA0
:100A2000FB007A08AC00AD01AD00AC017B08AC0462
:100A3000AD1F212D7116AC09AD09AC0A0319AD0A21
:100A4000222D71122D08F5002C08F4000530F60057
:100A5000F701E1277508A1007408A000210DA10C81
:100A6000A00C210DA10CA00C210DA10CA00CB1011A
:100A7000B001B2012108AB002008AA002B08803A7F
:100A8000FF0080307F02031D472D0A302A028312A7
:100A900003132A08031C692DF63EBA002B0803181D
:100AA000013EFF3EBB00BB1B5A2DF630B20AAA071F
:100AB000031CAB033208C925BB1B612D0A30B00AE9
:100AC000B2023008C925BB1B3E2D0A30B10AB00264
:100AD0003E2D8A267508A9007408A80032088A26C7
:100AE0007508A7007408A60030088A267508A500B6
:100AF0007408A40031088A267508A3007408A200AF
:100B0000711E862D9430A2008330A300B108031D0E
:100B10000800B008031DC12DB208031DB62D2B0817
:100B20002A04031DA32DB930A6008330A700A50019
:100B30002608A4002508A3002408A200D630A80097
:100B40008330A9000800711EA92D9430A4008330C1
:100B5000AC2DB930A4008330A500B930A200833099
:100B6000A300D630A6008330A7000800711EBC2D5C
:100B70009430A4008330BF2DB930A4008330A50089
:100B8000D02D711EC82D9430A2008330A300080020
:100B9000D02DF63EBA00FF3003180030BB0008002D
:100BA000B930A2008330A3000800C000203040020A
:100BB000031CEA2D7E3040020318EA2D400835263A
:100BC000E1277508BF007408BE006030BE07031C33
:100BD000BF03102EC03040024008031C002EFF3A15
:100BE0000319FF2D40083526E1277508BF0074085A
:100BF000BE006730BE070318BF0AFD300F2E400845
:100C0000FF3A031D080040083526E1277508BF009C
:100C10007408BE004030BE070318BF0AFC30BF078F
:100C20000530BC00BD018130831203133F07FF0074
:100C300012303E0784000318FF0A0021BA00BB01EE
:100C40002F20BE0A0319BF0AFF30BC07031CBD03D7
:100C50003D08803AFF0080307F02031D312E0130B5
:100C60003C020318132E00302F28F4000530F50144
:100C7000F600F7010800640083120313AF01AE0110
:100C800083160516051E482E8316031306154B2ED4
:100C9000831603130611831205120611831605121B
:100CA000061173200516051E592E8316031306150B
:100CB0005C2E8316031306116E2070118312061921
:100CC0007015F01183120313051AF01569207012C4
:100CD0008312031306197016F01283120313051AF8
:100CE000F016701A772E83120313AE01AE0AF01AB3
:100CF0007D2E83120313AF01AF0A701D832E831262
:100D00000313AE0AAE0AF01D892E83120313AF0A35
:100D1000AF0AFA2FF600BE2ED630F4008330F5006D
:100D20000800D830F4008330F5000800DA30F40011
:100D30008330F5000800DC30F4008330F500080053
:100D4000DE30F4008330F5000800E030F40083303A
:100D5000F5000800E230F4008330F5000800E430CC
:100D6000F4008330F5000800E630F4008330F5002D
:100D70000800E830F4008330F500080076088400AD
:100D80000A3004020318080000308A0045300407C6
:100D9000820008000830F600F50164008312031396
:100DA00005128316051200000000000083160313CD
:100DB0000516FA27F0108312051AF0146E2003109E
:100DC000F50CF01CE52E8030F507FA27F603031D1D
:100DD000CD2EFA27750808000830F600F5016400EA
:100DE0008312031306118316061100000000000091
:100DF000831603130615FA27701083120619701450
:100E00006E200310F50C701C072F8030F507FA27B1
:100E1000F603031DEF2EFA2775080800F5000830C9
:100E2000F600F0107518F0148312031305128316E0
:100E300005120000000000000000F01C232F8316A4
:100E400003130516262F8316031305126E200516AD
:100E5000FA270310F50CF603031D112FFA2FF500E6
:100E60000830F60070107518701483120313061101
:100E7000831606110000000000000000701C442FC3
:100E8000831603130615472F8316031306116E20CE
:100E90000615FA270310F50CF603031D322FFA2F5F
:100EA000F40064000830F500F60183120313061203
:100EB000F41F5C2F06145D2F0610FF30061603107A
:100EC000F40DF507031CF6037608803AFF00803026
:100ED0007F02031D6D2F01307502031C0800552F82
:100EE0006400831203138615861400008312031313
:100EF00086112020213086153A20C2303A20073052
:100F00003A2013303A2020303A2009303A20AD27D9
:100F100008303A200C303A200030F80158280730C9
:100F2000831203139F0086018501FF30831685001D
:100F3000C430860020308B0083128C0183168C0114
:100F400007308100F030831281008B17701371110C
:100F50007110F013F111F11008000030F801582061
:100F6000F830FA000130FB00640000302F20FF3021
:100F7000FA07031CFB037B08803AFF0080307F02E6
:100F8000031DC42F01307A02031C0800B42F8B1AF2
:100F90000B1DDA2FF0300B11831203138100B70AF7
:100FA000711CD52FB80FD52F7115F11CDA2FB90F81
:100FB000DA2FF11573088A00720E8300FE0E7E0E82
:100FC0000900F801F901741CEB2F7608F8070318E3
:100FD000F90A7708F9070310F60DF70D0310F50C61
:100FE000F40C75087404031DE32F7908F5007808E4
:0E0FF000F40008000230F400F40BFC2F08009F
:02400E003C3F35
:00000001FF
